:100000001E290408A2008316861383120930A30058
:1000100003101520A20CA30B09280314152003308C
:10002000A100E830C5200314192903181A2800007C
:1000300086171C2886131C280030A1006630C528AE
:10004000B71329080319B7170530A8002730A300F4
:10005000103036200330A300E8303620A30164308E
:100060003620A3010A30362024083D28A2002508A6
:10007000A1002408A000F8202008A000A80303196C
:10008000B713290803194728280203180800200875
:10009000031DB713B71B0800303E1429A3003A080C
:1000A000840038097E208413A30803191929F0302D
:1000B000A50022088038A400F030A5030319A5008C
:1000C0000319A303031919292008A6002108A70072
:1000D0002730C4202608A0002708A1009220030191
:1000E00020183808A21F3808A20803190301A40F1A
:1000F0007B28800659287C2800005C28841780050E
:100100001929A000A00DA00D200D3839C1389F007D
:100110000030A1003230C5201F151F198D28A10104
:100120001E081929210820040319A00A8030201A6A
:10013000A1062019A106A018A106210DA00DA10D50
:10014000192903178D0083168C130C1483120C08C5
:10015000192903178C0083168C130C1555308D004C
:10016000AA308D008C148C18B3280C111929A30106
:10017000A200FF30A207031CA307031C19290330A8
:10018000A100E630C520B928A101FC3EA000A109CC
:10019000031CD028FF300000A0070318CB28A007BD
:1001A0006400A10FCA280800A101A301A200023027
:1001B000E128A301A2000330E128A301A20004303A
:1001C000E128A80023082102031DE82822082002B4
:1001D000043003180130031902302805031DFF30D5
:1001E00019290038031DFF300405031DFF301929AC
:1001F000A501A4011030A600210DA40DA50D220813
:10020000A4022308031C230FA50203180E292208A9
:10021000A40723080318230FA5070310A00DA10DA1
:10022000A60BFC2820081929840031088A00300810
:1002300082008313031383126400080083160711DE
:100240005730920083122C3095000C309700043008
:1002500092008316EF308500C5308600203087007D
:1002600002309F00831286108316861083120612B6
:10027000831606128312861183168611203083128C
:100280008A01022020308A01022062308A01022085
:1002900069308A0102206C308A0102206C308A01A8
:1002A000022073308A01022062308A0102206F30FE
:1002B0008A01022074308A01022031308A01022032
:1002C00030308A0102202E308A01022062308A01F9
:1002D000022061308A01022073308A0102200A3034
:1002E0008A0102200D308A010220071083160710B0
:1002F0008312861283168612831287108316871044
:10030000831207138316071383128711831687112D
:100310008312071283160712003083128A01A1206C
:10032000CF0001308A01A120CA0064308A01B720C1
:100330000530BA001030B8007830A2000A308A01C7
:100340004E2064308A01B72064008A110A12061810
:10035000AC298A110A12432C861483168610640075
:100360008A110A1283120618AC2986108316861089
:1003700005308312BA001030B8005A30A2000A309B
:100380008A014E200330A300B6308A01B8208614BB
:100390008316861005308312BA001030B80064301E
:1003A000A2000A308A014E200130A300C2308A0127
:1003B000B82086108316861083120130A300F43013
:1003C0008A01B82086148316861005308312BA007D
:1003D0001030B8006E30A2000A308A014E20013081
:1003E000A300C2308A01B8208610831686108312BB
:1003F0000130A300F4308A01B820861483168610D9
:1004000005308312BA001030B8007330A2000A30F1
:100410008A014E200130A300C2308A01B820861024
:100420008316861083120130A300F4308A01B820AD
:1004300086148316861005308312BA001030B80077
:100440007830A2000A308A014E200130A300C23069
:100450008A01B82086108316861083120130A3000B
:10046000F4308A01B82086148316861083127830FF
:10047000C8008A110A12B9238A110A12852364302E
:100480008A01B7208A110A123C268A110A125323C4
:1004900006128316061283128611831686118312A2
:1004A0008A110A12B9230030871A0130A0000030E7
:1004B0008A01D420B200003006190130A0000030BB
:1004C0008A01D420B4003208840034088A01F12063
:1004D000B400B5006400340835048A110A12031907
:1004E000772A8A110A123A238A110A123C266400DA
:1004F0004908013C8A110A12031D812A8A110A1235
:10050000B22A64004908023C8A110A12031D8B2A90
:100510008A110A12E52A8A110A12B9230030871AB1
:100520000130A00000308A01D420B200003006194A
:100530000130A00000308A01D420B40032088400C9
:1005400034088A01F120B400B50064003408350491
:100550008A110A120319B22A8A110A123A238A113D
:100560000A123C268A110A12B9230030871A013078
:10057000A00000308A01D420B200003006190130FA
:10058000A00001308A01D420B4003208840034086D
:100590008A01F120B400B5006400340835048A11E2
:1005A0000A120319E52A06168316061283128A1107
:1005B0000A1285238A110A123C268A110A123A234A
:1005C0000130C9008A110A123C268A110A12B92385
:1005D000003006190130A00000308A01D420B2009A
:1005E0000030871A0130A00001308A01D420B40005
:1005F0003208840034088A01F120B400B500640098
:10060000340835048A110A120319182B861583162B
:10061000861183128A110A129E238A110A123C261D
:100620008A110A123A230230C9008A110A123C26A2
:100630000030871A0130A00001308A01D420B200B6
:10064000003006190130A00001308A01D420B40026
:100650003208840034088A01F120B400B500640037
:10066000340835048A110A120319382B8A01392AF1
:100670008A01482A87118316871183120716831669
:1006800007128312871083168710831207178316A9
:100690000713831286168316861283120714831695
:1006A000071083120800871183168711831207121F
:1006B000831607128312871083168710831207137D
:1006C0008316071383128616831686128312071465
:1006D000831607108312080087158316871183126B
:1006E000071283160712831287148316871083124A
:1006F0000713831607138312861683168612831236
:1007000007148316071083120800871583168711B4
:10071000831207128316071283128710831687101D
:100720008312071783160713831286168316861201
:10073000831207148316071083120800871183168B
:1007400087118312071683160712831287148316E4
:1007500087108312071383160713831286168316D6
:1007600086128312071483160710831208008A0169
:10077000392A00308A018120C6002108C7000130D3
:100780008A018120C2002108C3004608A000470852
:10079000A1004F088A01DD20B2004608A0004708EA
:1007A000A1004F088A01DD20B4003208840034081B
:1007B0008A01F120B400B5006400340835048A11C0
:1007C0000A120319F22B8A015323C8308A01B72079
:1007D0008A110A123C268A016C230230A300BC3025
:1007E0008A01B82000308A018120C6002108C70094
:1007F0004608A0004708A1004F088A01D9208A11A5
:100800000A12031D1A2C8A015323C8308A01B7200B
:100810008A110A123C268A016C230230A300BC30E4
:100820008A01B8208A019E230130A300F4308A0196
:10083000B820C90101308A018120C2002108C3000B
:100840004208A0004308A1004A088A01D9208A1161
:100850000A12031D422C8A015323C8308A01B72093
:100860008A110A123C268A016C230230A300BC3094
:100870008A01B8208A0185230130A300F4308A015F
:10088000B820C901080006128316061283128611C9
:1008900083168611831286108316861083122030E9
:1008A0008A01022063308A01022061308A0102201D
:1008B0006C308A01022069308A01022062308A018C
:1008C000022072308A01022061308A0102207430D5
:1008D0008A01022065308A01022020308A0102202C
:1008E00062308A0102206C308A01022061308A0164
:1008F000022063308A0102206B308A0102202030FE
:100900008A0102200A308A0102200D308A01022069
:1009100000308A018120CD0001308A018120CB0086
:100920008614831686108312061683160612053067
:100930008312BA001030B8006E30A2000A308A016B
:100940004E206C308A01022065308A010220663018
:100950008A01022074308A01022062308A0102205A
:100960006C308A01022061308A01022063308A01E2
:1009700002206B308A01022020308A010220A90166
:100980004B08A400A5010130B000B1018A0120206C
:1009900020308A01022072308A01022069308A01E7
:1009A000022067308A01022068308A0102207430F8
:1009B0008A01022062308A0102206C308A01022002
:1009C00061308A01022063308A0102206B308A0183
:1009D000022020308A010220A9014D08A400A501AF
:1009E0000130B000B1018A0120200A308A010220C2
:1009F0000D308A01022064008A110A12061CFB2CA9
:100A00000130A300F4308A01B82064008A110A1270
:100A1000061C0C2D8A01052D0530BA001030B800D7
:100A20006E30A2000A308A014E2000308A018120F7
:100A3000CE0001308A018120CC006C308A01022076
:100A400065308A01022066308A01022074308A01F2
:100A5000022077308A01022068308A010220693042
:100A60008A01022074308A01022065308A01022046
:100A700020308A010220A9014C08A400A501013000
:100A8000B000B1018A01202020308A01022072309A
:100A90008A01022069308A01022067308A0102201F
:100AA00068308A01022074308A01022077308A017E
:100AB000022068308A01022069308A0102207430E5
:100AC0008A01022065308A01022020308A0102203A
:100AD000A9014E08A400A5010130B000B1018A01AE
:100AE00020200A308A0102200D308A0102204E089F
:100AF0004D02B200B301031CB3030310B30CB20CDC
:100B00004E083207CF004C084B02B200B301031C61
:100B1000B3030310B30CB20C4C083207CA006C309C
:100B20008A01022065308A01022066308A01022093
:100B300074308A01022072308A01022065308A01F5
:100B4000022066308A01022020308A010220A90199
:100B50004A08A400A5010130B000B1018A0120209B
:100B600020308A01022072308A01022069308A0115
:100B7000022067308A01022068308A010220743026
:100B80008A01022072308A01022065308A01022027
:100B900066308A01022020308A010220A9014F0814
:100BA000A400A5010130B000B1018A0120200A3063
:100BB0008A0102200D308A01022064004E084F0293
:100BC0008A110A12031C282E64004C084A028A115A
:100BD0000A12031C282E03178D0103134F088A01E4
:100BE000A920031701308D0003134A088A01A920A8
:100BF000861583168611831286108316861005309B
:100C00008312BA001030B8006430A20014308A0198
:100C10004E2064308A01B7200530BA001030B80089
:100C20006430A20014308A014E2064308A01B7205B
:100C30000530BA001030B8006430A20014308A01C8
:100C40004E200130A300F4308A01B8208A01AC297B
:100C50000530BA001030B8006430A20014308A01A8
:100C60004E200530BA001030B8005030A2001430C9
:100C70008A014E208A01282E64008A110A12061C5D
:100C8000562E0530C80264004808503C8A110A12EA
:100C9000031D4C2E7D30C8000530BA001030B8005E
:100CA0004808A2000A308A014E2008008A01532316
:100CB000861083168610643083128A01B72086144A
:100CC00083168610643083128A01B7208A01562E5B
:02400E00723FFF
:00000001FF
